:020000040000FA
:020000002828AE
:080008002000111C0900111079
:10001000960197011C305A23AF002F1D272822007C
:100020009D012500930120000C191B2822008C1231
:100030000C1620001F2822000C128C1620002F1CEA
:10004000272820000C08303A22008C0020000900EC
:100050008C0123008C0121007A30990021000F309F
:100060008C002100111420002130980020000B1773
:100070008B1722009D141D1425000C3093002500C1
:10008000910108305A23AB00AB1D4B282000FF30F4
:100090009B002000502820007F309B00200050282B
:1000A00020000B302B059C008C01B301B7011D30E3
:1000B0005A23B000B0187828330803196F2801308C
:1000C0005A23A9003302031867282908B300043013
:1000D0005A23AA003302031C6F282A08B300AB1965
:1000E00073280310B30C2000330825009100200072
:1000F000A201A301A401A501A601A701A001A101DC
:100100000C1993280C199528003020020319802817
:100110002030200203189928A10A0C30210203196B
:100120009C28A00180280000000000000000A00A18
:100130008028A001A1018028A001A1010C19AC28F0
:100140000C19AE280030200203199E28203020020E
:100150000318B228A0019E28000000000000000043
:10016000A00A9E2896019701A001A101A1150C19D2
:10017000CA280C19CC28003020020319B7282030D7
:1001800020020318D028A20D2214A10BC828D428BD
:10019000A001B7280000000000000000A00AB72856
:1001A000A20D2210A10BC828A001A1010C19E4285E
:1001B0000C19E628003020020319D628203020022E
:1001C0000318EA28A00178280000000000000000C1
:1001D000A00AD628A001A101A1150C1900290C190B
:1001E0000229003020020319ED28203020020318D4
:1001F0000629A30D2314A10BFE280A29A001ED282E
:100200000000000000000000A00AED28A30D23104C
:10021000A10BFE28A001A1010C191A290C191C29F7
:100220000030200203190C29203020020318202955
:10023000A00178280000000000000000A00A0C299E
:10024000A001A101A1150C1936290C19382900307B
:100250002002031923292030200203183C29A40D71
:100260002414A10B34294029A001232900000000F7
:1002700000000000A00A2329A40D2410A10B34299A
:10028000A001A1010C1950290C195229003020029B
:10029000031942292030200203185629A001E2291F
:1002A0000000000000000000A00A4229A001A101F6
:1002B000A1150C196C290C196E29003020020319A4
:1002C00059292030200203187229A50D2514A10BED
:1002D0006A297629A00159290000000000000000C9
:1002E000A00A5929A50D2510A10B6A29A001A10179
:1002F0000C1986290C198829003020020319782945
:100300002030200203188C29A001E22900000000FF
:1003100000000000A00A7829A001A101A1150C1974
:10032000A2290C19A4290030200203198F2920309A
:1003300020020318A829A60D2614A10BA029AC2978
:10034000A0018F290000000000000000A00A8F29F2
:10035000A60D2610A10BA029A001A1010C19BC29F2
:100360000C19BE29003020020319AE2920302002CA
:100370000318C229A001E2290000000000000000CB
:10038000A00AAE29A001A101A1150C19D8290C19A8
:10039000DA29003020020319C52920302002031871
:1003A000DE29A70D2714A10BD629E229A001C52912
:1003B0000000000000000000A00AC529A70D2710BA
:1003C000A10BD62922082306240625062606270681
:1003D000031D78282209031DEF29B7017828220878
:1003E0000319422BA21B042A7039703A0319B72A49
:1003F000B7011C305A23AF00AF1A782800305A23B7
:100400002206031D78281E2AB7011C305A23AF008C
:10041000AF1E78282208193E0318782810305A2376
:100420002206031D782811305A232306031D78283D
:100430002408A3002508A4002608A5002308E03905
:10044000BA00203A03196A2A3A08803A0319912A15
:100450003A08E03A0319AA2A3A08003A0319422B4B
:100460003A08403A03193D2A3A08603A03193D2AEE
:100470003A08A03A0319A62A78281C305A23AF005C
:100480002F1C452A2308203AA300AF184E2A231E0A
:100490004D2AA31E4C2A4D2A4D2A23160314231E2F
:1004A000031023080F39B400B40DB41634085A23CE
:1004B000B3001C15A31A632A31143210250016103C
:1004C0009614200057283214311025009610161467
:1004D000200057283F302302031D78282408B3004A
:1004E000B3130310B30D20001C151C305A23AF00AA
:1004F0002F1C7D2A2408FF3AA400A41B882A31144B
:100500003210250016100000961400002000572815
:10051000321431102500961000001614000020003F
:1005200057281D305A23B00030189E2AB0189F2A31
:100530001C305A23AF00AF1C782878287828231E57
:10054000A42AFF30B3006F28B3016F28A31EA92A85
:1005500078287828EC302302031D782807302406F9
:100560000319652B2508B90024084A234128371CA4
:10057000F829A5080319FF2A2208783A0319C92A7D
:100580002208743A0319E72A22087C3A0319EF2A51
:100590007828241A782823085A23B800DA22B805C4
:1005A000A41DD62A3808031D90237828380803197B
:1005B0009023782802308A00240807398207013402
:1005C0000234043408341034203440348034230896
:1005D0005A232402031D7828B70190237828073076
:1005E0002306031DF82A08302406031D8D2B692BD2
:1005F0002408B90023084A23B70190237828221D34
:10060000102BA2187828221C2D2B062B2308B500AE
:10061000B5030310B50D0310B50DB714902378285A
:10062000B71C7828220803393507B600073036068C
:100630000319602BA21D242B2308B90036084A2376
:10064000B601B7019023782836085A232302031DE8
:100650007828B601B70190237828B71C7828A21D06
:10066000392B2308B9001C304A23B501B701902368
:1006700078281C305A232302031D7828B501B701BE
:100680009023782822082306031D78283714B30105
:100690008C01572823009100200039082300930083
:1006A000151555309600AA30960095149518562BBE
:1006B00020000800230091001514130820000800F2
:1006C00008302306031D8D2B692B08302506031DDA
:1006D00078280330B90000304A230030B9000130D7
:1006E0004A23FF30B90004304A230130B9000C30EE
:1006F0004A23C030B90010304A238030B90011308D
:100700004A230230B9001C304A230030B9001D30A2
:100710004A230030B90008304A23B501B701412807
:10072000CC309300FF30B3009100FF308C00A82341
:10073000A823A823A823A823A8238C01B3019101EF
:100740009301080000000C30BD00BD0BA52B080074
:100750005B30BE00A223AC2BBE0BAA2B000008000E
:0C0760003C30BF00A823BF0BB22B0800E8
:020000040001F9
:02000E00A40943
:02001000FF1CD3
:10E000000300000000000000FF0000001F009C0053
:10E0100000000000000000000100000000000000FF
:10E02000C0008000000000000000000000000000B0
:10E0300000000000000000000200000000000000DE
:10E040000000000000000000090012001B00240076
:10E050002E0037004000490052005B0064006D0054
:10E0600076008000890092009B00A400AD00B600FD
:10E07000BF00C800D100DB00E400ED00F600FF00A7
:00000001FF
